:1000000084EF5EF00000000000EF00F00000000050
:0A0010000000000000000000F3D71C
:10BD0800070EAF6EAC8479D8670E5D6E720E5E6EEC
:0EBD1800A0D8005202E0B4D801D04ED9FFD717
:10BD2600F2CF01F06DC0F6FF6EC0F7FF6FC0F8FFEF
:10BD3600A68EA69CA684A688F29E550EA76EAA0E6F
:10BD4600A76EA682F28E0A0071C0E9FF72C0EAFFF2
:10BD5600036A010E035C14E2026A400E025C05E20D
:10BD6600EECFF5FF0F00022AF8D7A68EA69CA68472
:10BD7600F29E550EA76EAA0EA76EA682032AE9D7D3
:0ABD8600F28EA69401C0F2FF120035
:0EBD9000ACB202D00000FCD760C0ADFF1200C4
:10BD9E00C00E00016D6FBF0E6E6F000E6F6F706F75
:10BDAE001D0E716F000E726FB7DF840E1D6EEF0EDB
:0CBDBE001E6E5E0E1F6EF00E206E120056
:0EBDCA00000E9EBA010E016E01C000F01200C4
:10BDD800AECF02F0ABA202D0AB98AB8802C001F0A4
:06BDE80001C000F0120092
:10BDEE00540E0C6E1C0E0D6E0D2EFED70C2EFCD7A7
:04BDFE00000012002F
:10BE0200900E196EBD0E1A6E600E1B6E000E1C6E29
:10BE1200D80E156EBD0E166E000E176E000E186E41
:10BE2200CA0E0001656FBD0E666F000E676F000ED1
:10BE3200686FFF0E616FFF0E626F000E636F000E80
:10BE4200646FAC8A900EAB6E948E949C9EAA03D0C3
:08BE5200AECF00F0FBD7120097
:10BE5A005F6AC8DF5DC060F096DFC4DF5F2A5F50AB
:10BE6A00FF0A02E15F6A08D0B2DF00505E1803E100
:0EBE7A00010E5F6E01D0EDD75FC000F0120028
:10BE88005D6A0001696B6A6B6B6B6C6B5D50400A95
:10BE980025E10001000E006E6C1908E100506B19D5
:10BEA80005E100506A1902E16951000A01E173DFF6
:10BEB80069C06DF06AC06EF06BC06FF06CC070F056
:10BEC8001D0E0001716F000E726F29DF5D6A400E52
:10BED80000016927000E6A236B236C230001790E89
:10BEE800606F52DF6EDF0050000AFCE071DF00C0B7
:10BEF8005FF0780E0001606F47DF63DF0050000AD3
:10BF0800FCE066DF00C05EF01D0EE16E000EE26E22
:10BF18005D50E126D8B0E22A5FC0E6FF5D2A1D0E1B
:10BF2800E16E000EE26E5D50E126D8B0E22A5EC0F6
:08BF3800E6FF5D2AABD7120001
:10BFC0000000000000000000000000000000000071
:10BFD0000000000000000000000000000000000061
:10BFE0000000000000000000000000000000000051
:0EBFF000000000000000000000000000120031
:020000040030CA
:0D00010006011EF38380FF07C007E00740E3
:00000001FF
